:10000000C20C02005F00F50C0500000C0600640045
:1000100084056000E403080A650066006C00080CB3
:100020002D00330069006A007100110501022B00E8
:1000300009028B00EA010B02290068000A0CAA00E1
:100040000307240AA8021F0AEA0128095109160A0F
:10005000640010024306350A080243060008B00097
:100060000307350A4306350A000870000304050734
:1000700003057103510700081102710011052B00DF
:100080002B03AB010B07000803042B0603057203C7
:10009000F30200080D023300120234002C05720036
:1000A0000008450600082C0700082C04140226004E
:0C00B00065050000000000006504000869
:04202000AA00F3001F
:00000001FF
